:100000002EC1189518951895189518951895189546
:10001000189518951895BCC01895189518951895A9
:1000200018951895189501007D0008006300680078
:100030006B006D00700074007600790001009D0077
:100040000800830088008B008D00900094009600CB
:1000500099000100BD000800A300A800AB00AD009E
:10006000B000B400B600B9000700A000000000E92D
:100070000AB90EE800BD00E000BD09E109B90FEFC3
:1000800007BB04BB0EEF01BB00E002BB0093A20064
:100090000093A000089504E1E0E5F3EC31971E2FF2
:1000A0001F2BE1F70A95C1F708954BD1902F11232B
:1000B00011F4822F02C089E0821B9923F1F4082FEA
:1000C000E6E2F0E0E9C0C098C19AC298C39A15C0B0
:1000D000C098C198FACFC09AFCCFC09AC1980BC003
:1000E000C09AC198C29A08C0C098FBCFC098C19A64
:1000F000F9CFC098C19AC298C3989130F1F4082FF3
:10010000ECE3F0E0C9C0A898A99AAA98AB9A15C0E8
:10011000A898A998FACFA89AFCCFA89AA9980BC03A
:10012000A89AA998AA9A08C0A898FBCFA898A99AB3
:10013000F9CFA898A99AAA98AB989230F1F4082F11
:10014000E2E5F0E0A9C09498959A9698979A15C020
:1001500094989598FACF949AFCCF949A95980BC05E
:10016000949A9598969A08C09498FBCF9498959AEB
:10017000F9CF9498959A9698979880E002C08BDF73
:1001800083950091A4008017D0F385DFE2E0DCC006
:10019000FA93EA932A931A930A932FB7E0EAF0E0CE
:1001A0000281002319F50CB107FBBEF406FB16F41F
:1001B00011E001C010E01083102F107319F400E05B
:1001C000018314C0102F1073103111F401E0F8CF27
:1001D0000073003259F402E0F3CF1381112319F4B4
:1001E000048311E01383028300E003832FBF09918E
:1001F00019912991E991F9911895A1D0A5EAB0E05A
:1002000000E0E5EAF0E0018332DF26C02C91109196
:10021000A0000091A10049DF0C9103950C930930D7
:1002200010F001E00C93E2EAF0E000810A9500830F
:1002300001E0E5EAF0E001830091A200002331F73C
:10024000E5EAF0E00181002339F000E001830CE0F1
:100250000CB95E9BFECF5E9A01E00C93EDCF0FE9E7
:100260000DBF00E00EBFC0E8D0E077D0002309F05A
:1002700084D0C3DF9CD09BC05FD0702D5DD0602D3B
:100280005BD0502D59D0402D57D0102C01FA54D0AE
:10029000202C52D0302C0895F5DF041B10E003C051
:1002A000EFDF041B150B20E030E005C0E5DF041B89
:1002B000150B260B370BE0F010FC1DC03DD0402D78
:1002C0003BD0E00FF11F0417100540E0240734076E
:1002D00078F446F4C895002D0024E22DF32DE01BA0
:1002E000F0090994E00FF11F27D0202C25D0302CE5
:1002F000E22DF32D099411F4BEF7ECCF31960EF0F8
:10030000319650E060E070E017D0402D4B3F68F030
:1003100079F34F3F41F04E3F21F00ED0702D0CD0BD
:10032000602D0AD0502D08D0402D041B150B260B34
:10033000370B11F3E8F2E2CFC89531960895BA93DE
:10034000AA939A938A93089599818881F0E00FB6D1
:10035000F894CE0FDF1F0FBE089501E0089520E04E
:1003600002D0E9F708952D9301501040202F212B42
:1003700008952591F8DFE9F7089588E690E0FC01FB
:1003800005911491FC013296A591B491FC0134962B
:1003900025913491422F432B19F0F901EADF01C076
:1003A000DEDF069610E08E36910748F308950000D0
:0403B0008895FECF5F
:00000001FF
